:020000040000FA
:04000000A7EF04F072
:08000800056ED8CF06F0E0CF31
:1000100007F00001E9CF0DF0EACF08F0E1CF09F0D9
:10002000E2CF0AF0D9CF0BF0DACF0CF0F3CF14F017
:10003000F4CF15F0FACF16F000C00FF001C010F0A9
:1000400002C011F003C012F004C013F09DA02CEF09
:1000500000F09EB074EF00F0A0A232EF00F0A1B269
:10006000ADEF00F00FC000F010C001F011C002F0C1
:1000700012C003F013C004F00E8E0DC0E9FF08C0DB
:10008000EAFF09C0E1FF0AC0E2FF0BC0D9FF0CC0C4
:10009000DAFF14C0F3FF15C0F4FF16C0FAFF0550D5
:1000A00007C0E0FF06C0D8FF10007550070B006EB8
:1000B0007530016E013201321F0E01160150772496
:1000C000E96E000E7820EA6E016A012A002A01D04A
:1000D0000136002EFDD7765203E00150EF1203D017
:1000E000011E0150EF16000C466AD8904634036A90
:1000F000330FE96E000E0320EA6EECCF74F0ED5280
:10010000EFCF73F073C075F0010E766E0F0E786E40
:10011000890E776ECADF73C075F0766A0F0E786E3F
:10012000920E776EC2DFD8904634036A210FE96ED3
:10013000000E0320EA6EECCF74F0ED52EFCF73F0B7
:1001400074C0B3FF73C0B2FFA0829E90D10ECF6E79
:100150009C0ECE6E9E9032EF00F0D8904634036A2B
:10016000330FE96E000E0320EA6EECCF74F0ED520F
:10017000EFCF73F073C075F0766A0F0E786E890E4C
:10018000776E93DF73C075F0766A0F0E786E920EFD
:10019000776E8BDF462A4550465C03E1A092A19220
:1001A00030D0D8904634036A330FE96E000E032036
:1001B000EA6EECCF74F0ED52EFCF73F073C075F0D0
:1001C000010E766E0F0E786E890E776E6EDF73C03D
:1001D00075F0766A0F0E786E920E776E66DFA192DA
:1001E000D8904634036A210FE96E000E0320EA6EB0
:1001F000ECCF74F0ED52EFCF73F074C0B3FF73C067
:10020000B2FFA19232EF00F08E0E006E5CC001F0E2
:100210005BC002F0036A015209E102C001F0026A08
:10022000080E005E015202E1006A08D0D89001BEBB
:1002300004D0023601360006F9D7019E9EEF03F086
:100240006750D8B471D0006E6B50D8B46DD0002612
:1002500004E3810E002668E204D07F0E005E64E3B2
:1002600063E068C06FF06C506F1A688E6C8E6A50D5
:100270006E02F4CF71F069506D02F4CF03F0F3CF4A
:1002800070F06E02F3507126F4507022000E0322BB
:100290006A506D02F3507126F4507022000E026A0B
:1002A0000322022268506E02F3507026F45003229B
:1002B000000E022268506D02F3500326F450022211
:1002C000000E016A01226A506C02F3507026F4504D
:1002D0000322000E0222012269506C02F350032611
:1002E000F4500222000E012268506C02F3500226E4
:1002F000F4500122002A01BE05D0703603360236C2
:1003000001360006000E70AE0AD0032A0222012236
:10031000015005E1025003E1035001E1002A6FBEE4
:10032000018E6FAE019E04D0006A016A026A036A00
:10033000000C5F50D8B4A5D06B6E6350D8B4A1D078
:100340006B5E05E37F0E6B26D8B09BD006D0810E86
:100350006B5ED8A096D0D8B494D06BC000F0016A80
:10036000026A036A6A6A60C069F0698E61C068F0F7
:1003700062C067F0190E6B6E6650675E0DE2010E8B
:10038000685E0AE2695E08E26A5E06E26A2A692A33
:10039000682A6650672628D06550685E12E2010E12
:1003A000695E0FE26A5E0DE26A2A692A6550682674
:1003B0006650672619E3682A17E1692A15E16A2A57
:1003C00013D064508009695E0EE2010E6A5E0BE292
:1003D0006A2A64508009692665506826E9E3692A1B
:1003E000E7E16A2AE5D703806B2E01D00BD0D890C5
:1003F0006736683669366A36D89003360236013673
:100400006C36BAD76CA006D0D890013202320332D3
:100410006C3202D0000635E06CBE1ED0D890673634
:10042000683669366A366650675E07E2010E685EB6
:1004300004E2695E02E26A5E1AE36550685E05E204
:10044000010E695E02E26A5E12E364508009695E31
:1004500003E2010E6A5E0BE3032A09E1022A07E1C7
:10046000012A05E1002A0DE001320232033260C0A8
:100470006BF064506B1A6BAE02D0018E06D0019EF9
:1004800004D0006A016A026A036AC6EF03F0800EB4
:10049000D8B2681A6D6A6E6A64C06CF068506C1AE3
:1004A0006350D8B4DCD06B6E006E6750D8B4E0D027
:1004B0006B5ED8B481D03DE368C071F0718E69C0C5
:1004C00070F06AC06FF06E6AD890713270326F321D
:1004D0006E326B2EF8D76CAE03D06D80DDD06D9090
:1004E0006B906D88EA6A660EE96EE9D06D986CBE15
:1004F0000AD06BA013D0713270326F326E32002A84
:10050000D8B4C5D00BD071BE0CD0D8906E366F3633
:10051000703671360006D8B4BAD0F5D76D8C6BD072
:100520006D9C64C06CF064AE02D0718EA9D0719ED7
:10053000A7D067C06BF067C000F063506B5E64C00B
:1005400071F0718E65C070F066C06FF06E6AD89001
:10055000713270326F326E326B2EF8D76CAE03D0C0
:100560006D829AD06D926B906D8AEA6A6A0EE96E1E
:10057000A6D06D9A6CBE0AD06BA013D071327032C7
:100580006F326E32002AD8B482D00BD071BE0CD03C
:10059000D8906E366F36703671360006D8B477D084
:1005A000F5D76D8E28D06D9E68C06CF068AE02D015
:1005B000718E66D0719E64D068C071F0718E69C012
:1005C00070F06AC06FF06CAE04D0719E6D8464D020
:1005D0006D946E6A6B90EA6A660EE96E70D06CBEBE
:1005E0001CD064C06CF06BA006D0713270326F32D8
:1005F0006E32002A4CE06EAE0BD06F2A09E1702AF1
:1006000007E1712A05E1713270326F32002A3FE052
:100610006DBC86D76DBEC7D71CD0800E711A71AE67
:1006200004D03AD068C06CF00AD064C06CF071524B
:1006300006E1705204E16F5202E1006A21D071BEFE
:1006400008D0D8906E366F3670367136002EF7D7D8
:100650001ED06CAE02D0718E13D0719E11D067C0C7
:1006600000F068C071F069C070F06AC06FF008D027
:1006700063C000F064C071F065C070F066C06FF0D8
:1006800071C001F070C002F06FC003F034D0006A96
:10069000016A026A036A2FD06E6A6F1E701E711E95
:1006A0006E1E6E2A05E16F2A03E1702A01E1712AAC
:1006B0006DB015D76DB256D76DB48AD7B3D7EF509A
:1006C0006F2605E3702A03E1712AD8B46B80ED52DE
:1006D000EF50702603E3712AD8B46B80ED52EF50CF
:1006E000EFBE01D0800A7126D8B06B806DB8FED6FF
:1006F0006DBA3FD774D7E0EF03F08E0E006E6750EF
:10070000005E68C002F069C001F0028E005209E08C
:10071000D890025202E1015204E002320132002E6E
:10072000F7D768AE05D0011E021E012AD8B4022AEE
:1007300002EF04F05C6A5AC05BF066D503C06AF051
:1007400002C069F001C068F000C067F06F0E6E6E05
:10075000120E6D6E030E6C6E750E6B6E71DD00C049
:100760005BF001C05CF002C05DF003C05EF003C04E
:1007700062F002C061F001C060F000C05FF0666A24
:10078000656A7F0E646E860E636ED3D500C05FF01F
:1007900001C060F002C061F003C062F0D89203C0F3
:1007A00066F002C065F001C064F000C063F06F0E37
:1007B0006A6E120E696E030E686E750E676E67D6EE
:1007C00000C063F001C064F002C065F003C066F0D1
:1007D00003C06AF002C069F001C068F000C067F0B1
:1007E000800E6E6E960E6D6E180E6C6E930E6B6EA6
:1007F00027DD03C06AF002C069F001C068F000C0E4
:1008000067F07BD702C003F00150FF08006EFF0EB7
:10081000035600C001F003C002F0000C55C045F0C3
:10082000466A566A5550565C32E2D8905634036A8E
:100830005324E96E54500320EA6EECCF58F0ED5289
:10084000EFCF57F0575202E158521FE0D89056347C
:10085000036A330F016E000E032203C058F0D890D4
:100860005634036A5324E96E54500320EA6EECCFE9
:1008700003F0ED52EFCF59F058C0EAFF01C0E9FF95
:1008800003C0ECFFED5259C0EFFF562ACBD7566A92
:100890004550565C2BE2036A5650180FE96E000E65
:1008A0000320EA6E7F0EEF6ED8905634036A210F54
:1008B000016E000E032201C057F003C058F0036A16
:1008C0005650180FE96E000E0320EA6EEFCF59F074
:1008D00059C05AF02FDF58C0EAFF57C0E9FF02C0E5
:1008E000ECFFED5201C0EFFF562AD2D7B50ECD6E08
:1008F000D10ECF6E9C0ECE6EB150480BA509B16ED5
:100900009D80A092C00EF212FAEF04F0036A5450D8
:10091000180FE96E000E0320EA6E53C0EFFFD89067
:100920005434036A210F016E000E032201C055F0FA
:1009300003C056F053C05AF0FDDE56C0EAFF55C062
:10094000E9FF02C0ECFFED5201C0EFFF000CF86AB6
:10095000D09E0D8EEA6AE96A0A0EAF6EA60EAC6EE4
:10096000900EAB6EC180C182C184C196186A196AAB
:100970001A6A1B6A1C6A1D6A1E6A1F6A206A216A3B
:10098000226A236A246A256A266A276A286A296AEB
:100990002A6A2B6A2C6A2D6A2E6A2F6A306A316A9B
:1009A000326A336A346A356A366A376A386A396A4B
:1009B0003A6A3B6A3C6A3D6A3E6A3F6A406A416AFB
:1009C000426A436A446A456A080E476E7C0E486E66
:1009D000090E496E7C0E4A6E120E4B6E7C0E4C6EEA
:1009E000150E4D6E7C0E4E6E546A470E536E040EFD
:1009F000556E14D79EAAFED7AECF4FF09EAAFED753
:100A0000AECF50F09EAAFED7AECF51F09EAAFED731
:100A1000AECF52F04FC053F0546A78DF50C053F05D
:100A2000010E546E73DF51C053F0020E546E6EDF30
:100A300052C053F0030E546E69DF590E9EA8FED7C4
:060A4000AD6ED8D70300E3
:020000040030CA
:0E00000000220E0E000181000FC00FE00F4025
:00000001FF
